:100000000C949D020C94E1020C94E1020C94E10228
:100010000C94E1020C94E1020C94E1020C94E102D4
:100020000C94E1020C94E1020C941C120C94EE125C
:100030000C948D240C94E1020C94E1020C94E102E6
:100040000C94E1020C94E1020C94E1020C94E102A4
:100050000C94E1020C94FA240C94E1020C94E10259
:100060000C94E1020C94E1020C94E1020C94E10284
:100070000C94E1020C94E1020C94E1020C94E10274
:100080000C94860A0C94E1020C94E1020C94E102B7
:100090000C94E1020C94E1020C94E1020C94E10254
:1000A0000C94E1020C94E1020C94E10207634236E5
:1000B000B79BD8A71A39685618AEBAAB558C1D3CF9
:1000C000B7CC5763BD6DEDFD753EF6177231BF00BD
:1000D0000000803F08000000BE922449123EABAAF7
:1000E000AA2ABECDCCCC4C3E00000080BEABAAAA52
:1000F000AA3E00000000BF000000803F000000009A
:1001000000084178D3BB4387D1133D190E3CC3BDD2
:100110004282AD2B3E68EC8276BED98FE1A93E4C7F
:1001200080EFFFBE01C4FF7F3F0000000000000021
:10013000F1A4F1A3018C028C048C2B0014001A0092
:100140000800150017001C0018000C001200130016
:100150002A00290004001600070009000A000B000D
:100160000D000E000F0033003400E1001D001B00E5
:100170000600190005001100100036003700380095
:1001800028000030E000E200E30002202C002C00F8
:1001900001205000510052004F002B0014001A00A3
:1001A000090013000A000D000F0018001C003300A6
:1001B0002A002900040015001600170007000B0094
:1001C000110008000C0012003400E1001D001B00AB
:1001D0000600190005000E00100036003700380038
:1001E00028000030E000E200E30002202C002C0098
:1001F00001205000510052004F002B003400360007
:10020000370013001C0009000A00060015000F004B
:100210002A00290004001200080018000C00070042
:100220000B001700110016003800E1003300140025
:100230000D000E001B00050010001A0019001D0023
:1002400028000030E000E200E30002202C002C0037
:1002500001205000510052004F0035021E021F02C3
:100260002002210222022302240225022602270262
:100270002A0001003A003B003C003D003E003F00E8
:100280002D022E022F0230023102010040004100F7
:100290004200430044004500032004200520005094
:1002A0000100010001000100010002200100010025
:1002B0000100AB00AA00A900AE0035001E001F001F
:1002C0002000210022002300240025002600270012
:1002D0002A0001003A003B003C003D003E003F0088
:1002E0002D002E002F0030003100010040004100A1
:1002F0004200430044004500032004200520005034
:1003000001000100010001000100010001000100E5
:100310000120AB00AA00A900AE0028035400680029
:100320006500200050006C0061006E0063006B00EF
:1003300020004B006500790062006F0061007200D0
:10034000640000002C034F007200740068006F000E
:100350006C0069006E0065006100720020004B00B7
:100360006500790062006F00610072006400730034
:100370000000040309040902D000060100A03209AC
:100380000400000103010100092111010001223FC5
:10039000000705810308000A0904010001030102A6
:1003A00000092111010001224D0007058203080008
:1003B0000A090402000103000000092111010001E3
:1003C0002236000705830308000A0904030002031C
:1003D000000000092111010001222000070584030B
:1003E00020000107050403200001090404000001A6
:1003F00001000009240100010900010509040500AC
:10040000020103000007240100014100062402014B
:100410000100062402020200092403010301020173
:10042000000924030204010101000905060240003D
:1004300005000005250101010905850240000500B0
:100440000005250101031201100100000008EDFE66
:1004500060600100010200010631FF0974A1010979
:1004600075150025FF952075088102097615002570
:10047000FF952075089102C005010980A101850240
:1004800016010026B7001A01002AB7007510950161
:100490008100C0050C0901A1018503160100269CFD
:1004A000021A01002A9C02751095018100C0050105
:1004B0000902A1010901A100050919012905150079
:1004C00025019505750181029501750381010501DD
:1004D000093009311581257F950275088106093893
:1004E0001581257F950175088106050C0A380215CE
:1004F00081257F950175088106C0C005010906A107
:1005000001050719E029E715002501950875018106
:1005100002950175088101050819012905950575E0
:100520000191029501750391010507190029FF1535
:100530000025FF950675088100C011241FBECFEF6E
:10054000DAE0DEBFCDBF04B603FE24C0809178039D
:1005500090917903A0917A03B0917B038730904BFF
:10056000A740B04BB9F4109278031092790310921F
:100570007A0310927B0314BE84B7877F84BF88E11F
:100580000FB6F89480936000109260000FBEE0E018
:10059000F8E3099511E0A0E0B1E0E2EAFFE502C06E
:1005A00005900D92A63BB107D9F713E0A6EBB1E099
:1005B00001C01D92A837B107E1F70E94F90E0C9413
:1005C000CF2F0C9400000895089561110DC0FC0117
:1005D0008281882331F085EE0E949D190E94B62BFE
:1005E00003C085EE0E94651A80E090E008958B3B81
:1005F000910568F4883A910530F5853A9105C0F483
:100600008430910598F4019709F06FC071C0803E65
:10061000910508F46AC0883E910540F09C01205F76
:1006200031092031310508F060C05CC09C01A1C0D7
:10063000853A910509F45FC0863A910509F45EC0D8
:1006400023E830E496C0883A910509F45AC0893A03
:10065000910509F459C08A3A910509F458C08B3ABA
:10066000910509F457C08C3A910509F456C08D3AAA
:10067000910509F455C0803B910509F454C08E3AA8
:10068000910509F453C08F3A910509F452C0813B9A
:10069000910509F451C0823B910509F450C0833B98
:1006A000910509F44FC0843B910509F44EC0853B88
:1006B000910509F44DC0863B910509F44CC0873B78
:1006C000910509F44BC0883B910509F44AC0893B68
:1006D000910509F449C08A3B910509F048C02AE216
:1006E00036E447C09C01306544C020E030E041C0A2
:1006F00021E030E03EC021E830E43BC022E830E4B5
:1007000038C022EE34E435C029EE34E432C02AEE9B
:1007100034E42FC025EB34E42CC026EB34E429C0AC
:1007200027EB34E426C02CEC34E423C02DEC34E475
:1007300020C023E835E41DC02AE835E41AC022E9C8
:1007400035E417C024E935E414C021E236E411C0D1
:1007500023E236E40EC024E236E40BC025E236E4A0
:1007600008C026E236E405C027E236E402C020E0F5
:1007700034E4C90108959CE0799FF001112490E3CD
:10078000899FE00DF11D1124E60FF11DEE0FFF1FF3
:10079000E65CFE4F25913491C9010895880F991F99
:1007A00082559040FC0125913491C9010895880F2C
:1007B000991F825D9E4FFC0125913491C9010895D6
:1007C0000E94BB039C013A9521153F4108F4DFC00C
:1007D0009C0130522115304120F49F700E94D703B4
:1007E00008959C0130532115304118F49927906CDD
:1007F00008959C0130542031310520F48F709927E1
:10080000946D0895803120E4920719F480E091ED11
:100810000895813140E4940719F480E090ED089543
:10082000823120E4920719F480E092ED089583313B
:1008300040E4940719F480E093ED0895811520E5D4
:10084000920711F40C941F25813040E5940731F490
:100850008091680281608093680208959C013056FF
:100860002115304108F402C097FF02C0906F08952F
:10087000803E9105E0F4803C910568F58133910557
:1008800009F474C048F48932910509F46AC08A32C7
:10089000910509F07AC074C089339105F9F0823866
:1008A0009105E1F08533910509F06FC050C0833E9A
:1008B0009105A9F140F4803E9105C9F0823E910571
:1008C00009F063C01BC0863E910571F1873E91051A
:1008D00009F05BC037C00E94CE03089520917B02CF
:1008E00020FD02C021FF51C080EE90E04EC08091FB
:1008F0007B0280FFF9CF89E390E047C080917B02C3
:1009000082FF0AC080917B0284FF03C080E090E0F8
:100910003CC083EE90E039C082EE90E036C080911A
:100920007B0282FFEFCFF8CF80917B0283FF07C06D
:1009300080917B0284FDEACF87EE90E026C086EEB0
:1009400090E023C080917B0283FFF2CFF8CF8091AB
:100950007B0285FF03C089E290E017C085E390E049
:1009600014C080917B0285FDF9CFF5CF80917B0289
:1009700086FF03C08AE290E008C081E390E005C0F2
:1009800080917B0286FDF9CFF5CF0E94F702089592
:100990005F926F927F928F929F92AF92BF92CF920F
:1009A000DF92EF92FF920F931F93CF93DF93CDB718
:1009B000DEB728970FB6F894DEBF0FBECDBF9E01FD
:1009C0002F5F3F4F4E0189E0880E911C60E070E080
:1009D00000E010E0E12CF12CC12CD12CA12CB12C89
:1009E00088E0782E622E532E41E050E0E3E2F1E001
:1009F000A62DB52D872D01900D928A95E1F7F9016D
:100A0000819191919F01FC01E07FFF27E032F10588
:100A100059F48F709927FA0102C0EE0FFF1F8A95D3
:100A2000E2F7AE2ABF2A37C0E033F10559F48F70E0
:100A30009927FA0102C0EE0FFF1F8A95E2F7CE2A2E
:100A4000DF2A29C0E034F10559F48F709927FA01A3
:100A500002C0EE0FFF1F8A95E2F7EE2AFF2A1BC0A5
:100A6000E035F10559F48F709927FA0102C0EE0FB5
:100A7000FF1F8A95E2F70E2B1F2B0DC0E036F10504
:100A800051F48F709927FA0102C0EE0FFF1F8A956B
:100A9000E2F76E2B7F2B2815390509F0A7CF94B10B
:100AA0008A2D8095892384B985B18A2985B997B122
:100AB0008C2D8095892387B988B18C2988B99AB102
:100AC0008E2D809589238AB98BB18E298BB99DB1E2
:100AD000802F809589238DB98EB1802B8EB990B3EC
:100AE000862F8095892380BB81B3862B81BB289676
:100AF0000FB6F894DEBF0FBECDBFDF91CF911F912F
:100B00000F91FF90EF90DF90CF90BF90AF909F90AC
:100B10008F907F906F905F9008955F926F927F9219
:100B20008F929F92AF92BF92CF92DF92EF92FF92FD
:100B30000F931F93CF93DF93CDB7DEB768970FB6B0
:100B4000F894DEBF0FBECDBF85B7806885BF85B77F
:100B5000806885BF0E94CF076E9A769A0E94C8046B
:100B60009E012F5F3F4F4E0189E1880E911C60E08E
:100B700070E000E010E0E12CF12CC12CD12CA12C74
:100B8000B12C98E1792E622E532E41E050E0EBE239
:100B9000F1E0A62DB52D872D01900D928A95E1F7F4
:100BA000F901819191919F01FC01E07FFF27E032E3
